:020000040800F2
:10000000000002209D0200082F1100083111000895
:1000100033110008351100083711000800000000F6
:10002000000000000000000000000000391100087E
:100030003B110008000000003D1100083F110008BE
:10004000A90F0008A90F0008A90F0008A90F0008B0
:10005000A90F0008A90F0008A90F0008A90F0008A0
:10006000A90F0008A90F0008A90F0008A90F000890
:10007000A90F0008A90F0008A90F0008A90F000880
:10008000A90F0008A90F0008A90F0008A90F000870
:10009000A90F0008A90F0008A90F0008A90F000860
:1000A000A90F0008A90F0008A90F0008A90F000850
:1000B000A90F0008A90F0008A90F0008A90F000840
:1000C000A90F0008A90F0008A90F0008A90F000830
:1000D000A90F0008A90F0008A90F0008A90F000820
:1000E000A90F0008A90F0008A90F0008A90F000810
:1000F000A90F0008A90F0008A90F0008A90F000800
:10010000A90F0008A90F0008A90F0008A90F0008EF
:10011000A90F0008A90F0008A90F0008A90F0008DF
:10012000A90F0008A90F0008A90F0008A90F0008CF
:10013000A90F0008A90F0008A90F0008A90F0008BF
:10014000A90F0008A90F0008A90F0008A90F0008AF
:10015000A90F0008A90F0008A90F0008A90F00089F
:10016000A90F0008A90F0008A90F0008A90F00088F
:10017000A90F0008A90F0008A90F0008000000003F
:10018000A90F0008A90F000800B583B000F082FE97
:10019000304B314A1360314A1360314B314A03E02E
:1001A00011681960043304322F498B42F8D32A4B6B
:1001B0001A682E4B9A4200D0FEE7284B1A682C4B47
:1001C0009A42F9D1234B2B4A13602B4A13602B4BD5
:1001D00002E000221A600433294A9342F9D3254BE6
:1001E0001B6813B9244B1B6803B1FEE700F05EFEE9
:1001F000694601A800F02AFE224B234CE41AA41001
:100200000025AC4214DC214B214CE41AA41000253B
:10021000AC4213DC0099019800F085FF05461D4BA8
:100220001D4CE41AA410002C0EDC284600F0EAFD58
:10023000144B53F8253098470135E2E7134B53F838
:10024000253098470135E3E7013C124B53F8243041
:100250009847E8E7BABADECA000000207400002020
:10026000000000202C1C0008780000207856341272
:100270003254769878000020140100207800002085
:1002800018010020C8030008C8030008C8030008BC
:10029000C8030008C8030008C803000808B5FFF732
:1002A00073FF00BEFEE71EF0040F0CBFEFF30880E3
:1002B000EFF309807146374A10472DE9F04182B0CB
:1002C00004468846084B5E6B9F6B9D6A074800F0AA
:1002D000C5FDCDF800803B4632462946204600F059
:1002E000E9FD00BEFEE700BF00ED00E08C1B00084A
:1002F00000BEFEE71EF0040F0CBFEFF30880EFF323
:1003000009807146244A10472DE9F04182B0044625
:100310008846084B5E6B9F6B9D6A074800F09EFD08
:10032000CDF800803B4632462946204600F0C2FD0B
:1003300000BEFEE700ED00E09C1B00081EF0040F6D
:100340000CBFEFF30880EFF309807146134A1047A2
:100350002DE9F04182B004468846084B5E6B9F6BE6
:100360009D6A074800F07AFDCDF800803B46324692
:100370002946204600F09EFD00BEFEE700ED00E0AD
:10038000A81B000800BEFEE700BEFEE700BEFEE7B9
:1003900070470000BB020008090300085103000871
:1003A0002C1C000800000020780000202C1C0008F5
:1003B000000000100000001078000020180100204C
:0803C000000000100000001015
:1003D00010B50446074B1868074BA3FB0030800993
:1003E00000F04CF8002221464FF0FF3000F014F8E6
:1003F000002010BD0C000020D34D6210024A13688B
:1004000001331360704700BF0C010020014B1868D6
:10041000704700BF0C01002030B4164BDB68C3F3FB
:100420000223C3F10704042C28BF04241D1D062D3C
:1004300017D9033B012505FA04F4013C21409940FA
:1004400005FA03F3013B1340194300280BDB0901B4
:10045000C9B200F1604000F5614080F8001330BC83
:1004600070470023E6E700F00F000901C9B2024B14
:100470001954F4E700ED00E014ED00E00138B0F1AC
:10048000807F0AD2064B5860F021064A82F823107A
:100490000020986007221A6070470120704700BF53
:1004A00010E000E000ED00E0024B186800F4C060CE
:1004B000704700BF0070004030B583B00546204B48
:1004C0009B6D13F0805F0BD0FFF7EEFFB0F5007F60
:1004D00017D0802D1FD82DD0702D2DD000211BE0DE
:1004E000174CA36D43F08053A365A36D03F08053B5
:1004F0000193019BFFF7D8FFA36D23F08053A36501
:10050000E4E7802D03D9A02D03D9022104E00021C6
:1005100002E0012100E003210A4A136823F00703E7
:100520000B431360136803F00703994206D00120C0
:1005300003B030BD0221EFE70121EDE70020F7E72E
:10054000001002400020024010B4534B9B6813F08F
:100550000C0F1AD0504B9B6803F00C030C2B0ED0E1
:100560004D4B9B6803F00C03042B3DD04A4B9B681A
:1005700003F00C03082B3AD0002004461FE0464B42
:10058000DB6803F00303012BEAD1434B1B6813F034
:10059000080F1CD1404BD3F8943003F470634FF430
:1005A000706292FAA2F2B2FA82F2D3403B4A52F857
:1005B0002340394B9B6813F00C0F13D00020364AB0
:1005C000936803F00C030C2B14D010BC7047324B13
:1005D0001B6803F0F003F02292FAA2F2B2FA82F260
:1005E000D340E3E72046EAE72D480024E7E72D481B
:1005F0000024E4E7D16801F00301D36803F070033D
:10060000702292FAA2F2B2FA82F2D34001330229A6
:1006100011D003292FD0B4FBF3F31F4AD06800F4A4
:10062000FE404FF4FE4292FAA2F2B2FA82F2D040B9
:1006300000FB03F00FE01A48B0FBF3F3164AD06852
:1006400000F4FE404FF4FE4292FAA2F2B2FA82F2B5
:10065000D04000FB03F0104BDB6803F0C0634FF0A9
:10066000C06292FAA2F2B2FA82F2D34001335B0086
:10067000B0FBF3F0A9E70B48B0FBF3F3064AD068F0
:1006800000F4FE404FF4FE4292FAA2F2B2FA82F275
:10069000D04000FB03F0DEE700100240C81B00085A
:1006A0000024F40000127A0070B582B0044603689A
:1006B00013F0100F45D09B4B9B6813F00C0F40F0CC
:1006C0009880984B1B6813F0020F03D08369002BAE
:1006D00000F0AD82206A934B1B6813F0080F68D0BE
:1006E000904B1B6803F0F003834269D2FFF7E4FEEE
:1006F000002840F09E828B4B1A6842F008021A6074
:100700001A6822F0F002216A0A431A605A6822F439
:100710007F42E16942EA01225A60FFF715FF814BEF
:100720009B6803F0F003F02292FAA2F2B2FA82F28E
:10073000D3407D4AD35CD8407C4B18600F20FFF734
:1007400047FE236813F0010F00F0A180754B9B68F2
:1007500003F00C03082B00F09180724B9B6803F0B0
:100760000C030C2B00F083806368B3F5803F00F02E
:10077000B680B3F5A02F00F0B8806A4B1A6822F457
:1007800080321A601A6822F480221A606368002B93
:1007900000F0B880FFF73AFE0546624B1B6813F481
:1007A000003F74D1FFF732FE401B6428F5D90320C7
:1007B00046E25C4BD3F894301B0903F0F00393E757
:1007C000584B1A6842F008021A601A6822F0F002C8
:1007D000216A0A431A605A6822F47F42E16942EAB8
:1007E00001225A60206AFFF767FE002895D0012099
:1007F00026E2836933B34B4A136843F00103136065
:10080000FFF704FE0546474B1B6813F0020F06D1A5
:10081000FFF7FCFD401B0228F5D9032010E2414BF5
:100820001A6842F008021A601A6822F0F002216A7F
:100830000A431A605A6822F47F42E16942EA0122BF
:100840005A607EE7374A136823F001031360FFF70D
:10085000DDFD0546334B1B6813F0020F3FF471AF0B
:10086000FFF7D4FD401B0228F4D90320E8E12D4B0B
:10087000DB6803F00303032B7FF476AF294B1B687F
:1008800013F4003F03D06368002B00F0D481236889
:1008900013F0020F6AD0234B9B6803F00C03042B68
:1008A0004CD0204B9B6803F00C030C2B40D0E3682A
:1008B000002B00F089801B4A136843F48073136097
:1008C000FFF7A4FD0546174B1B6813F4806F6BD12F
:1008D000FFF79CFD401B0228F5D90320B0E1114A27
:1008E000136843F48033136050E703F18043A3F5AA
:1008F0003C331A6842F480221A601A6842F480324B
:100900001A6043E7FFF782FD0546064B1B6813F4A8
:10091000003FBCD0FFF77AFD401B6428F5D90320C7
:100920008EE100BF00100240B81B00080C00002040
:10093000A34BDB6803F00303022BB8D1A04B1B6869
:1009400013F4806F03D0E368002B00F076819C489D
:10095000436823F0F85321694FF0F85292FAA2F25B
:10096000B2FA82F201FA02F213434360236813F0F1
:10097000080F54D06369002B3AD0914AD2F89430D2
:1009800043F00103C2F89430FFF740FD05468C4B5D
:10099000D3F8943013F0020F41D1FFF737FD401B1D
:1009A0000228F4D903204BE18548436823F0F8532B
:1009B00021694FF0F85292FAA2F2B2FA82F201FAE9
:1009C00002F213434360D1E77D4A136823F4807336
:1009D0001360FFF71BFD0546794B1B6813F4806F0E
:1009E000C4D0FFF713FD401B0228F5D9032027E1EF
:1009F000734AD2F8943023F00103C2F89430FFF721
:100A000005FD05466E4BD3F8943013F0020F06D067
:100A1000FFF7FCFC401B0228F4D9032010E12368F7
:100A200013F0040F7BD0664B9B6D13F0805F36D1C3
:100A3000634B9A6D42F080529A659B6D03F0805330
:100A40000193019B01255F4B1B6813F4807F28D025
:100A5000A368012B39D0052B3FD0594BD3F89020F8
:100A600022F00102C3F89020D3F8902022F0040273
:100A7000C3F89020A368002B3DD0FFF7C7FC0646C3
:100A80004F4BD3F8903013F0020F46D1FFF7BEFC66
:100A9000801B41F288339842F2D90320D0E0002530
:100AA000D1E7484A136843F480731360FFF7AEFC44
:100AB0000646444B1B6813F4807FC9D1FFF7A6FCA0
:100AC000801B0228F5D90320BAE03D4AD2F89030C5
:100AD00043F00103C2F89030CCE7394BD3F89020B3
:100AE00042F00402C3F89020D3F8902042F00102B3
:100AF000C3F89020BEE7FFF789FC0646304BD3F8D9
:100B0000903013F0020F08D0FFF780FC801B41F2F9
:100B100088339842F2D9032092E0002D35D1A36AA0
:100B2000002B00F08C80264A926802F00C020C2AFE
:100B300000F08880022B2ED0214B1A6822F08072A0
:100B40001A601B6813F0006F09D11D4B1B6813F06E
:100B5000005F04D11A4AD36823F00303D360184A14
:100B6000D36823F0887323F48033D360FFF74EFCFF
:100B70000446134B1B6813F0007F56D0FFF746FC6A
:100B8000001B0228F5D903205AE00D4A936D23F08B
:100B900080539365C3E70A4A136823F08073136098
:100BA000FFF734FC0546064B1B6813F0007F0BD0A3
:100BB000FFF72CFC401B0228F5D9032040E000BFC2
:100BC0000010024000700040236B5A1E636B1B0232
:100BD00043EA0213A26B120943EA4243E26A134357
:100BE000E26B5208013A43EA4253226C5208013A3E
:100BF00043EA4263144AD360136843F0807313607E
:100C0000D36843F08073D360FFF700FC04460E4BBB
:100C10001B6813F0007F06D1FFF7F8FB001B0228CA
:100C2000F5D903200CE000200AE0002008E00120B4
:100C300006E0012004E0012002E0012000E00020A5
:100C400002B070BD0120FBE700100240694B1B6839
:100C500003F007038B420CD2664A136823F00703A4
:100C60000B431360136803F00703994201D001207E
:100C7000704770B5036813F0020F06D05E4A9368A0
:100C800023F0F0038468234393600C460546036811
:100C900013F0010F6CD04368022B0AD0032B2DD028
:100CA000002B32D1544A126812F0020F07D10120F2
:100CB00070BD514A126812F4003F00F099804E490D
:100CC0008A6822F0030213438B60FFF79FFB0646FE
:100CD0006B68022B20D0032B2DD0002B3AD0464B33
:100CE0009B6803F00C03042B42D0FFF78FFB801BA3
:100CF00041F288339842F2D9032070BD3E4A12680F
:100D000012F0007FDBD1012070BD3B4A126812F463
:100D1000806FD4D1012070BD374B9B6803F00C036A
:100D2000082B25D0FFF772FB801B41F288339842D5
:100D3000F2D9032070BD304B9B6803F00C030C2BE1
:100D400016D0FFF763FB801B41F288339842F2D93B
:100D5000032070BD284B9B6813F00C0F08D0FFF7E1
:100D600055FB801B41F288339842F3D9032070BDB4
:100D7000204B1B6803F007039C420CD21D4A1368EA
:100D800023F0070323431360136803F007039C4217
:100D900001D0012070BD2B6813F0040F06D0164A55
:100DA000936823F4E063E9680B4393602B6813F0C6
:100DB000080F07D0104A936823F46053296943EA67
:100DC000C1039360FFF7C0FB0B4B9B6803F0F0037C
:100DD000F02292FAA2F2B2FA82F2D340074AD35C2E
:100DE000D840074B18600F20FFF7F2FA002070BDC3
:100DF000012070BD0020024000100240B81B000816
:100E00000C000020FEE7000008B503460C4A1268FB
:100E10005AB10B4A1068033323F003030344094A11
:100E2000934206D8064A136008BD0749044A116078
:100E3000EFE700F089F90C2303604FF0FF3008BDA5
:100E40007C00002000FC0120180100200123036029
:100E5000014B0B60704700BF040000200FB400B5C9
:100E600083B004AB53F8042B01938021064800F0B3
:100E7000B1F9002803DD0146034800F007F803B08C
:100E80005DF804EB04B07047840000204FF0FF30A1
:100E90007047000008B500F089F8024B024A9A60DA
:100EA00008BD00BF00ED00E00000000808B500F03C
:100EB0009BF808BDF8B504460D4617461E46274860
:100EC000FFF7CCFF21682648FFF7C8FF6168254877
:100ED000FFF7C4FFA1682448FFF7C0FFE16823487B
:100EE000FFF7BCFF21692248FFF7B8FF616921487D
:100EF000FFF7B4FFA1692048FFF7B0FFE1691F4881
:100F0000FFF7ACFF1E48FFF7A9FF29461D48FFF772
:100F1000A5FF1D4CE16A1D48FFF7A0FF216B1C488F
:100F2000FFF79CFFE16B1B48FFF798FF15F0800F60
:100F30000AD115F4004F0CD11748FFF78FFF06991F
:100F40001648FFF78BFFF8BD39461548FFF786FFB7
:100F5000EFE731461348FFF781FFEDE7701A00080D
:100F6000801A0008901A0008A01A0008B01A000899
:100F7000C01A0008D01A0008E01A0008F01A000889
:100F8000001B00080C1B000800ED00E01C1B000803
:100F90002C1B00083C1B00086C1B0008741B00087D
:100FA0004C1B00085C1B0008FEE700000C4B1A6895
:100FB00042F001021A60002199601A6822F0A852DA
:100FC00022F410221A604FF48052DA601A6822F478
:100FD00080221A6099614FF00062024B9A6070475C
:100FE0000010024000ED00E02F4B1B6813F0080FCB
:100FF00016D12D4BD3F89430C3F303232B4A52F868
:101000002320294B9B6803F00C030C2B48D8DFE806
:1010100003F00C474747194747471D4747472100FB
:10102000214B1B68C3F30313E8E7214B1A601E4BE7
:101030009B68C3F303131F4AD15C1D4A1368CB405E
:10104000136070471C4A1A4B1A60F0E71B4A184B92
:101050001A60ECE7144BD96801F00301DB68C3F3B5
:1010600002130133022904D0032915D0B2FBF3F295
:1010700002E0114AB2FBF3F20B49CB68C3F306233B
:1010800003FB02F3CA68C2F3416201325200B3FBB0
:10109000F2F3074A1360CAE7084AB2FBF3F2EBE740
:1010A000034B1A60C3E700BF00100240C81B0008D2
:1010B0000C000020B81B00080024F40000127A0085
:1010C00000B597B0002111911291139114911591CF
:1010D0004422684600F049F8102300930123069348
:1010E0006022089202220A920B930C9328230D93FC
:1010F000109207230E9304230F936846FFF7D4FA48
:1011000000B1FEE70F2311930323129300231393DF
:1011100014931593042111A8FFF798FD00B1FEE781
:1011200017B05DF804FB08B5FFF7CAFFFEE770478C
:10113000FEE7FEE7FEE7FEE770477047704708B539
:10114000FFF75CF908BD0000014B1868704700BF4D
:101150001000002010B5431E0A44914200D110BD7A
:1011600011F8014B03F8014FF7E70244034693429D
:1011700000D1704703F8011BF9E730B5141E05468E
:101180009BB0184605DA8B232B604FF0FF301BB065
:1011900030BD4FF40273ADF80C3014BF04F1FF33CF
:1011A0002346029305934FF6FF7300910491ADF827
:1011B0000E3002461E9B6946284600F075F8431C17
:1011C000BCBF8B232B60002CE1D0009B00221A7047
:1011D000DDE7000007B5009313460A4601460348C1
:1011E0000068FFF7CAFF03B05DF804FB10000020A1
:1011F0002DE9F0478E689E4282460C4691469846FD
:1012000035D88A8912F4906F31D0256809696F1A30
:101210006569022305EB450595FBF3F508F101032C
:101220003B449D4238BF1D46530531D5294600F049
:101230007FFB064650B90C23CAF80030A38943F05F
:101240004003A3814FF0FF30BDE8F0873A462169A3
:10125000FFF780FFA38923F4906343F08003A38109
:10126000266165613E44ED1B2660A5604646464505
:1012700028BF464632464946206800F0F1FAA36886
:101280009B1BA36023681E4426600020BDE8F087F6
:101290002A4600F0ABFB06460028E1D12169504602
:1012A00000F0F8FAC7E700002DE9F04F9DB0804646
:1012B00003938B891C060D4616460FD50B696BB937
:1012C000402100F035FB2860286128B90C23C8F8BC
:1012D00000304FF0FF30C5E040236B6100230993DD
:1012E00020238DF8293030238DF82A304FF0010B60
:1012F00037463C4614F8013B002B3CD1B7EB060ABD
:101300000BD05346324629464046FFF771FF013065
:1013100000F0A380099B534409933B78002B00F015
:101320009C8000234FF0FF320493079305920693AD
:101330008DF853301A9305222178504800F040FA76
:10134000671C049BD8B9D90644BF20228DF85320CE
:101350001A0744BF2B228DF8532022782A2A16D050
:10136000079A00210A20274601343B78303B092B9D
:1013700051D9C9B111E0252BC0D02746B9E73F4A62
:10138000801A0BFA00F0184304903C46D3E7039A06
:10139000111D12680391002A01DB079204E05242FA
:1013A00043F00203079204933B782E2B0ED17B78F7
:1013B0002A2B07F1010132D1039B1A1D1B680392EE
:1013C000002BB8BF4FF0FF33023705932C4C397810
:1013D0000322204600F0F4F938B14023001B03FA41
:1013E00000F0049B034304930137397825488DF8B6
:1013F000281006227E1C00F0E3F9002835D0224B8D
:10140000FBB9039B073323F0070308330393099BBE
:101410004B4409936CE700FB02320121A3E7002350
:10142000059318460A240F4601313A78303A092AC2
:1014300003D9002BCAD00590C8E704FB0020012384
:10144000F1E703AB00932A46104B04A94046AFF3E3
:101450000080B0F1FF3F8146D9D1AB895B063FF5F3
:1014600038AF09981DB0BDE8F08F03AB00932A4652
:10147000064B04A9404600F081F8EAE7F81B000893
:10148000FE1B0008021C000800000000F11100080B
:101490002DE9F04791461F468A680B69DDF82080E8
:1014A0009342B8BF1346C9F8003091F8432006466E
:1014B0000C4612B10133C9F800302368990642BFC7
:1014C000D9F800300233C9F80030256815F0060558
:1014D00007D104F1190AE368D9F800209B1A9D424C
:1014E00029DB94F843302268003318BF01239206A9
:1014F0002ED404F1430239463046C047013021D092
:101500002368E568D9F8002003F00603042B08BF20
:10151000AD1AA36822690CBF25EAE5750025934240
:10152000C4BF9B1AED184FF000091A344D451BD16A
:101530000020BDE8F0870123524639463046C047B7
:10154000013003D14FF0FF30BDE8F0870135C2E72D
:10155000E1185A1C302081F84300224494F84510C9
:1015600082F843100233C4E701232246394630464D
:10157000C0470130E6D009F10109D7E72DE9F04372
:1015800017460A7E85B06E2A984606460C460C9B86
:1015900001F1430E00F0BC801AD8632A2ED00AD87D
:1015A000002A00F0C880582A00F08A8004F1420521
:1015B00084F842202AE0642A01D0692AF6D1216801
:1015C0001A6811F0800F23D0111D1960136827E0ED
:1015D000732A00F0B48008D86F2A2AD0702AE5D187
:1015E0000A6842F020020A6003E0752A21D0782AB6
:1015F000DCD1782284F845206E4964E01A6801F154
:101600004205111D1960136884F842300123A3E0DC
:1016100011F0400F02F104011960D7D0B2F9003087
:10162000002B03DA2D225B4284F8432062490A2210
:1016300017E02068196810F0800F03D0081D1860AB
:101640000B6806E010F0400F01F104001860F7D0BD
:101650000B8859496F2A14BF0A220822002084F8F7
:1016600043006568A560002DC0F29C80206820F0D2
:1016700004002060002B3FD1002D40F0958075467E
:10168000082A0BD12368DA0708D5236962689A42D1
:10169000DEBF302305F8013C05F1FF35AEEB050355
:1016A0002361CDF800803B4603AA21463046FFF770
:1016B000EFFE013055D14FF0FF3005B0BDE8F083AB
:1016C00081F845203C492268186812F0800F00F12B
:1016D00004051D6001D0036802E05506FBD50388B0
:1016E000D00744BF42F0200222601BB9226822F0DA
:1016F000200222601022B1E77546B3FBF2F002FB34
:101700001033CB5C05F8013D03460028F5D1B7E75F
:1017100008681A68496910F0800F04D0101D18601D
:101720001368196007E010F0400F02F10400186020
:101730001368F6D01980002323617546B1E71A6853
:10174000111D1960156862680021284600F038F8FC
:1017500008B1401B606063682361002384F8433054
:101760009FE723692A4639463046C0470130A2D058
:1017700023689B0707D5002504F11909E368039A3C
:101780009B1A9D4205DBE068039B9842B8BF184650
:1017900093E701234A4639463046C04701308AD094
:1017A0000135EBE7002BA7D10B7884F8423004F128
:1017B000420565E71A1C0008091C0008000000002B
:1017C00001F0FF01102A2BDB10F0070F08D010F8F2
:1017D000013B013A8B422DD010F0070F42B3F6D1F6
:1017E000F0B441EA012141EA014122F007047FF00F
:1017F00000070023F0E80256083C85EA010586EA66
:10180000010685FA47F5A3FA87F586FA47F6A5FAA1
:1018100087F68EB9EED1F0BC01F0FF0102F00702AD
:1018200032B110F8013B013A83EA010313B1F8D158
:101830000020704701387047002D06BF3546033839
:10184000073815F0010F07D1013015F4807F02BF72
:10185000013015F4C03F0130F0BC0138704700BFC3
:10186000884210B501EB020303D8421E99420CD105
:1018700010BD9842F9D28118D21AD34200D110BDBE
:1018800013F8014D01F8014DF7E711F8014B02F88B
:10189000014FEBE738B50546002945D051F8043C27
:1018A0000C1F002BB8BFE41800F0D6F81F4A1368CD
:1018B000104633B9636014602846BDE8384000F034
:1018C000CCB8A3420CD921686218934204BF1A68AD
:1018D0005B68636004BF521822600460ECE7134643
:1018E0005A680AB1A242FAD919685818A0420BD115
:1018F00020680144581882421960DDD1106852688E
:101900005A6001441960D7E702D90C232B60D3E752
:10191000206821188A4204BF11685268626004BFBF
:10192000091821605C60C7E738BD00BF04010020D2
:1019300070B5CD1C25F0030508350C2D38BF0C25DE
:10194000002D064601DBA94203D90C233360002099
:1019500070BD00F081F8234A1468214691B9224CE9
:1019600023681BB9304600F067F8206029463046EE
:1019700000F062F8431C26D10C233360304600F09F
:101980006CF8E4E70B685B1B1AD40B2B0FD90B60C8
:10199000CD50CC18304600F060F804F10B00231D48
:1019A00020F00700C31A1BD05A42E25070BD8C428F
:1019B0000DBF63684B686360136018BF0C46E9E7AE
:1019C0000C464968CAE7C41C24F00304A04205D0B1
:1019D000211A304600F030F80130CDD02560D9E72B
:1019E00070BD00BF0401002008010020F8B50746C3
:1019F00014460E4621B91146BDE8F840FFF798BFDE
:101A000022B9FFF747FF25462846F8BD00F026F823
:101A100084420FD921463846FFF78AFF0546002841
:101A2000F2D031462246FFF795FB31463846FFF7A4
:101A300031FFE9E73546E7E738B5064C00230546B0
:101A400008462360FFF7E0F9431C02D1236803B185
:101A50002B6038BD100100207047704751F8040C0E
:101A60000028A0F10400BCBF0B58C018704700004C
:101A7000537461636B206672616D653A0A00000001
:101A8000205230203D2020253038580A0000000028
:101A9000205231203D2020253038580A0000000017
:101AA000205232203D2020253038580A0000000006
:101AB000205233203D2020253038580A00000000F5
:101AC00020523132203D20253038580A00000000D5
:101AD000204C52203D2020253038580A00000000BC
:101AE000205043203D2020253038580A00000000B7
:101AF00020505352203D20253038580A0000000065
:101B00004653522F4641523A0A00000020434653A2
:101B100052203D2020253038580A000020484653E6
:101B200052203D2020253038580A000020444653DA
:101B300052203D2020253038580A000020414653CD
:101B400052203D2020253038580A0000204D4D46B7
:101B50004152203D20253038580A0000204246419D
:101B600052203D2020253038580A00004D6973630B
:101B70000A000000204C522F4558435F52455455EF
:101B8000524E3D20253038580A0000005B486172F3
:101B9000644661756C745D0A000000005B427573F9
:101BA0004661756C745D0A005B55736167654661DB
:101BB000756C745D0A000000000000000000000069
:101BC0000102030406070809A0860100400D030076
:101BD000801A060000350C0040420F0080841E0071
:101BE00000093D0000127A000024F40000366E0166
:101BF0000048E801006CDC02232D302B2000686CCB
:101C00004C0065666745464700303132333435361F
:101C10003738394142434445460030313233343558
:0B1C2000363738396162636465660086
:101C2C0078563412800000200000000000093D00AE
:101C3C001400002000000000000000000000000064
:101C4C000000000000000000000000000000000088
:101C5C000000000000000000000000000000000078
:101C6C000000000000000000000000000000000068
:101C7C000000000000000000000000000000000058
:101C8C000000000000000000000000000000000048
:081C9C000000000032547698AC
:040000050800018965
:00000001FF
